:040000008A01032846
:0600060000008A11A62F84
:100F4C00F50183018A11C22FF1000430F3005330F4
:100F5C00F2000130F202031DB42FB52FAF2F013078
:100F6C00F302031DBA2FBB2FAD2F0130F102031D6D
:100F7C00C02FC12FAB2F0800981307308316031313
:100F8C009C0003100030031801309D00031000304A
:100F9C00031801309B001E3085000310003003182D
:100FAC000130860003100030031801308312031344
:100FBC00860005100130F4007408831203138607B1
:100FCC0083120313851CEB2FEC2FF92F0514C8305B
:100FDC008A11AA278A11831203130510C8308A11AB
:100FEC00AA278A11E62F14308A11AA278A11E02F1A
:040FFC008A1104282A
:00000001FF
